:020000040000FA
:10000000850186018316063085008601831207303C
:020010009F004F
:0A001600A2010519112885182428FD
:100020000B281920051D0B282C20221C3A287E2085
:100030000B28CE30AA000830AB00AA0B2028AB0B4F
:100040001D282228000008001920851C0B282C20C0
:10005000221C532893200B284F30A000C430A1004D
:10006000A00B3328A10B3028352805192214851838
:10007000221408008615051D3A2843204B204320F2
:100080004B2043206C288518722805194328192015
:1000900005194328080085187228051D4B281920CA
:1000A000051D4B2808000616851C53285C2064207B
:1000B0005C2064205C206F280519782885185C284E
:1000C000192085185C28080005197828851C6428E3
:1000D0001920851C6428080005196C2872288518C9
:1000E0006F2878288611A301A401A5017E200B2882
:1000F0000612A301A401A50193200B2805197E284F
:100100000330A6001830A7000230A800A60B8928EB
:10011000A70B8B28A80B86288D288E288F280519D9
:100120007E28A2010800851893280330A600183005
:10013000A7000230A800A60B9E28A70BA028A80B9A
:100140009B28A228A328A42885189328A201080088
:00000001FF
